:020000020000FC
:100000001FC039C23AC23FC23FC23FC23BC23FC219
:100010003FC23FC23FC23FC23FC22EC22FC22FC209
:0600200030C22EC233C203
:10004000F89400E812E008BD18BD11E00EE51EBFEF
:100050000DBF00E00BBB0CEF0ABB00E808BB0FE7CD
:1000600007BBB0E0A0E6D1E0C0E600E00D93BD170D
:10007000E9F7AC17D9F700E006BF00E00BBF00E0DE
:1000800009BF00EE0ABF0FEF08BF00E005BF00E0A8
:1000900005BB00E003BF00E003BB00E002BB10E0D3
:1000A00000E015BD0DBD00E015BD0CBD00E015BDA7
:1000B0000BBD00E015BD0ABD00E000BF00E00FBDB4
:1000C00000B7007F006007BD00E006BD00E000B99A
:1000D00000E009BD04B7086104BF09E601BD00E006
:1000E0000FB900E00EB900E00DB900E808B900E072
:1000F00009B900E007B905E806B900E103B903E072
:1001000001B900E002B900E00BBF00E009BF90E0D8
:1001100007E003E007E007E207E00FEF36D3C698F9
:10012000C59800000000000000000000000000E38F
:100130000BBB000000000000000000000000C49A9B
:10014000000000000000000000000000C49805E06E
:100150001CD300E30BBB0000000000000000000007
:100160000000C49A00000000000000000000000031
:10017000C49805E00AD300E30BBB000000000000B8
:10018000000000000000C49A000000000000000011
:1001900000000000C49805E0F8D200E20BBB0000AC
:1001A00000000000000000000000C49A00000000F1
:1001B0000000000000000000C49805E0E6D200E264
:1001C0000BBB000000000000000000000000C49A0B
:1001D000000000000000000000000000C49805E0DE
:1001E000D4D200E80BBB00000000000000000000BB
:1001F0000000C49A000000000000000000000000A1
:10020000C49805E0C2D20CE09BD105E0BED201E06B
:1002100097D103E0BAD206E093D10AEFB6D20AEF43
:10022000B4D2A895C09A01E0B0D200E003B900E0D2
:1002300007B933D11093600000936100C098C29A4F
:10024000C19A01E0A2D2C19800E803B90BE007B956
:1002500024D1C29810936200009363001091620051
:10026000009163003AE228EFB0D13093640020930C
:100270006500109366000093670010916000009184
:10028000610030E02AE0A1D110936800009369007A
:100290001091680000916900309162002091630024
:1002A000021B130B10936A0000936B0030916400E3
:1002B00020916500109166000091670070E060E099
:1002C00050916A0040916B009BD130936C00209359
:1002D0006D0010936E0000936F001091620000910A
:1002E00063001130D9F40F3FC9F400E20093080114
:1002F0000FE40093090106E500930A0105E4009369
:100300000B0102E500930C0100E200930D010DE6E4
:1003100000930E0104EF00930F0141C000916200B1
:1003200001FF19C000E20093080100E200930901F7
:1003300000E200930A0100E300930B010EE2009338
:100340000C0100E300930D010DE600930E0104EF94
:1003500000930F0124C010916E0000916F0099D19D
:10036000403351F440E2303339F430E2203321F4A9
:1003700020E2103309F410E250E250930801409358
:10038000090130930A0120930B0110930C01009393
:100390000D015DE650930E0154EF50930F01C09A8A
:1003A00001E0F3D100E003B900E007B976D0109383
:1003B0007000009371001091700000917100133073
:1003C000D9F40F3FC9F400E2009300010FE4009359
:1003D000010106E50093020105E40093030102E533
:1003E0000093040100E20093050100E2009306017E
:1003F00006E50093070135C010917000009171006F
:100400003CE126EBE2D0309372002093730010930E
:1004100074000093750070E060E05BEB41EDF0D09C
:100420003093760020937700109378000093790042
:1004300030D1203309F420E250E25093000150E221
:100440005093010150E25093020120930301109355
:1004500004015EE2509305010093060156E55093B6
:1004600007014DD00AEF91D10AEF8FD10AEF8DD15C
:100470000AEF8BD1D6CE1895189518951895189522
:100480001895189518951895189518951895189504
:10049000189518951895189518952F9320E026B95A
:1004A00025EC26B926B126FDFDCF04B115B12F915B
:1004B0000895DF01A07F1D911C91103029F409E0FF
:1004C000602E01E0702E1AC0113029F409E0602E70
:1004D00009E0702E13C0123029F407E0602E09E005
:1004E000702E0CC0133029F403E0602E0FE1702E43
:1004F00005C001E0602E04E0702E00C008951F9337
:10050000B1E0A0E000E000681BD018E00D911BD026
:100510000000000000000000000000001A95B1F784
:1005200000E400680DD018E00D910DD0000000002F
:1005300000000000000000001A95B1F71F91089517
:10054000C69804D00895C69A01D008951F932F939A
:10055000C5980000000000000000000000001BB370
:100560001F70202F207F122B1BBB000000000000FB
:10057000000000000000C49A00000000000000001D
:1005800000000000C498000000000000000000000F
:1005900000001BB31F70202F220F220F220F220FEB
:1005A000122B1BBB00000000000000000000000038
:1005B000C49A000000000000000000000000C49881
:1005C00005E0E3D02F911F9108954F935F936F93B0
:1005D000551B441B61E110F4400F511F579547957F
:1005E000379527956A95B9F75F934F933F932F936C
:1005F0000F911F912F913F916F915F914F910895AE
:100600008F939F93AF93BF93CF9388279927AA2760
:10061000BB27C0E2000F111F221F331F881F991F25
:10062000AA1FBB1F84179507A607B70728F00395D5
:10063000841B950BA60BB70BCA9561F7CF91BF91A1
:10064000AF919F918F9108950F931F932F933F9395
:10065000021B130B3F912F911F910F9108951F9330
:1006600010E3010F1F9108953F9334E620E0239596
:10067000031BE8F72A95030F3AE010E01395031BDC
:10068000E8F71A95030F30E3230F130F030F3F9181
:1006900008955F936F9367E250E140E04395051B37
:1006A000160BE0F74A95050F161F63E058EE30E091
:1006B0003395051B160BE0F73A95050F161F60E002
:1006C00054E620E02395051B160BE0F72A95050F4D
:1006D000161F5AE010E01395051BE8F71A95050F51
:1006E00050E3450F350F250F150F050F6F915F91E3
:1006F00008954F935F936F934427552760E1000F50
:10070000111F441F551F4217530718F00395421B32
:10071000530B6A95A1F75F934F932F913F916F9180
:100720005F914F9108956F937F938F939F93662767
:100730007727882798E1000F111F221F661F771F58
:10074000881F63177407850720F00395631B740BDC
:10075000850B9A9581F79F918F917F916F91089565
:100760001F93E199FECF10E01CBB5FBB4EBB0DBBDE
:10077000653A11F4E29AE19A1F910895E199FECF4A
:100780005FBB4EBBE09A0DB308951F932F932AE0F1
:1007900013E41A95F1F72A95D9F70A95C1F72F9125
:0407A0001F91089508
:00000001FF
